:0200000021F4E9
:1D000300C000C0E07422254E254EF8C2AF864C08864DD2AFD203D0E0D000C2A8327C
:0200230021C1F9
:20002B00C2CFC0E0C0F0C082C083C0D0752100E5227008E52370047C000192D208E52A1521
:20004B002A7044E518C39CFB50027B00E5237007E518C395225001E4F5F0C39BEB4002E513
:20006B00F08510F0A4252EF52AE522700215231522BCFF027CFE0CE5322536F536540725A2
:20008B003A90043993F548E5247008E52570047D0001EBD209E52B152B7045E519C39DFBDD
:2000AB0050027B00E5257007E519C395245001E4F5F0C39BEB4002E5F08511F0A4252FF580
:2000CB002BE524700215251524BDFF027DFE0DE5332537F5375407253B90043993C4F549F9
:2000EB00E5267008E52770047E002143D20AE52C152C7044E51AC39EFB50027B00E527708A
:20010B0007E51AC395265001E4F5F0C39BEB4002E5F08512F0A42530F52CE526700215277C
:20012B001526BEFF027EFE0EE5342538F5385407253C90043993F54AE5287008E52970042B
:20014B007F00219CD20BE52D152D7045E51BC39FFB50027F00E5297007E51BC395285001EE
:20016B00E4F5F0C39BEB4002E5F08513F0A42531F52DE528700215291528BFFF027FFE0F61
:20018B00E5352539F5395407253D90043993C4F54BE521700A20B707E4F580F5A0800CE5D0
:2001AB00484549F580E54A454BF5A0D0D0D083D082D0F0D0E03230982FC0E0C0D0C298A786
:2001CB009930000AB74207200216D2028947300207B70D04C202D20109430180EAB501045C
:2001EB00D2B380FED0D0D0E03275800075A000758E0175814F758780758922E5B0C45407CC
:20020B0090043193F58DF58BD288D28E759852784E760018B801FAD2007A8079807402F529
:20022B0010F511F512F5137432F514F515F516F51775CBFE75CA8E75C80475A8B075B82058
:20024B00C2B3515B517B71FC80F8515B3000FB22EAB50101223099FDC2998A008699C20079
:20026B00B60D02D2000A4302802285F047C20122200101220547434780A847E6C394304014
:20028B00E9F546940950E3753F078547F00547434780A847E6C3943040D0940A50CCD53F58
:2002AB00EC85F0477545070547434780A847E6C39430C0E0E545243DF8D0E0F6D545E8E568
:2002CB004175F00AA42540F540E54375F00AA4254275F064A42540F540E435F0F541E53F19
:2002EB0075F00AA4253EF53EE544F54254062323F543E544540175440160037544FFE54694
:20030B00B40021E514C3952E5001E48510F084C2CA854022854123853E2E85433A854432F6
:20032B00F51861D7B40121E515C3952F5001E48511F084C2CA854024854125853E2F8543BD
:20034B003B854433F51961D7B40221E516C395305001E48512F084C2CA8540268541278592
:20036B003E3085433C854434F51A61D7B40321E517C395315001E48513F084C2CA854028A5
:20038B00854129853E3185433D854435F51B61D7B4040585409061D7B4050471ED61D7B4D3
:2003AB00060985424EC289D2A861D7B40717434203E5422410F8E53E6016A63EE542241488
:2003CB00F8A64061D7B4080871DE61D7D2CAB2B3C20122515574429129E521911E740D91EE
:2003EB002922515574429129E5909114740D912922300314515574429129E54D9114E54CB5
:20040B009114740D9129C20322C0E0C4911ED0E0911E22540FB40A004002240724303099CB
:20042B00FDC299F59922FFFEFDFAF4E8D0A003060C0903060C0901030206040C08090102FD
:0E044B0004080102040801020408010204086A
:00000001FF
